:100000000C9488000C9460020C94A5000C94A5003C
:100010000C94A5000C94A5000C94A5000C94A500CC
:100020000C94A5000C94A5000C94A5000C94A500BC
:100030000C94A5000C94A5000C94A5000C94A500AC
:100040000C94A5000C94A5000C94A5000C94A5009C
:100050000C94A500040309042203770077007700BD
:100060002E00630072007900700074006F006D0054
:10007000790073002E00640065001E0356002D00F9
:100080005500530042002D004D0049004400490036
:100090002D0044004200470012011001000000083A
:1000A000C016E40501000102000109026500020119
:1000B0000080320904000000010100000924010051
:1000C00001090001010904010002010300000724E5
:1000D000010001410006240201010006240202027F
:1000E00000092403010301020100092403020401A1
:1000F0000101000905010308000A000005250101AE
:10010000010905810308000A00000525010103001B
:1001100011241FBECFE5D4E0DEBFCDBF10E0A0E6C6
:10012000B0E0E8E0FAE002C005900D92A237B10716
:10013000D9F710E0A2E7B0E001C01D92AA3AB107DA
:10014000E1F70E9422040C9402050C94000085B78C
:10015000836085BF8BB780648BBF8BE48093800006
:100160008AE580937F0008951F93DC01162F80910C
:100170007F008E3171F180917F0084FF07C08091F4
:10018000800098E889278093800003C08AE58093E7
:100190007F00912FE1E8F0E08D9181939150191645
:1001A000DCF381E890E0612F0E945C021C5F6FE746
:1001B00070E010937F00CB0123E0959587952A95F9
:1001C000E1F7837011508F5D6F5F7F4F412F0E9469
:1001D0009D031F9108951F93CF93DF93409190004B
:1001E000142F135017FDD8C080918D00CCE0D0E0C3
:1001F000C81BD109CC56DF4F80918C008F704150C5
:10020000805FBE010E949D0380918C00803128F4A4
:10021000CE01612F0E941204BDC08D3209F0A8C02A
:10022000183009F0B7C083EC809374008AE580939E
:100230006000109272009881892F807629F0CE019B
:100240000E94EE03282F81C02A813C8110927D00FC
:100250008981882381F49F71923049F4313839F4CF
:1002600080917F008E3119F481E080937D0010929F
:100270007E0022E063C0813011F0833089F42223B4
:1002800009F05BC0313809F058C0813011F08EE1BF
:1002900001C08AE580937F008BE4809380004DC08D
:1002A000853019F42093910048C0863079F58B8110
:1002B000813011F0823029F4CE010E94DA03282F18
:1002C00021C08330F1F4222341F484E590E090933F
:1002D0008F0080938E0024E015C0213041F488E522
:1002E00090E090938F0080938E0022E20BC022302A
:1002F00041F48AE790E090938F0080938E002EE186
:1003000001C020E080E4809372001FC0883021F497
:1003100021E083E990E014C0893019F42093930020
:1003200009C08A3011F421E009C08B3031F48BE42C
:10033000809380008AE580937F0020E08DE790E045
:1003400090938F0080938E0009C02F3F39F48881ED
:1003500087FD2E8180E88093720006C08F818823FC
:1003600019F46E81621708F0622F6093610012C069
:100370008091720087FF0EC0CE01612F0E940C0495
:100380008F3F21F48EE18093600004C0882311F038
:1003900010926100109290008091600084FF60C014
:1003A000809161008F3F09F45BC0182F893008F0FD
:1003B00018E0811B809361008091740098E8892780
:1003C00080937400112399F18091720087FF09C016
:1003D00085E790E0612F0E94FE03182F8930A0F579
:1003E00026C020918E0030918F0086FF0DC0A5E7BA
:1003F000B0E080E090E0F901E80FF91FE491ED939F
:1004000001961817C1F708C0912FD901E5E7F0E070
:100410008D9181939150E1F71150812F90E01F5FF2
:100420000196820F931F90938F0080938E0085E733
:1004300090E0612F0E945C02412F4C5F4C3041F0F4
:100440008FEF8093610004C08FEF809361004EE1D5
:1004500040936000415080E264E770E00E949D0399
:1004600094E180B38C7079F49150D9F71092910097
:1004700010928B008AE580937F008FEF60E070E040
:1004800040E00E949D03DF91CF911F910895A82F16
:10049000B92F80E090E041E050EA60956F5F58F43A
:1004A0002D9138EF82279795879510F0842795270F
:1004B0003F5FC8F3F3CF0895EADF8D939D930895CE
:1004C000CF93CFB7CF93C395839BE9F7839B09C0A5
:1004D000839B07C0839B05C0839B03C0839B01C094
:1004E000A6C0DF93C0918D00DD27CC56DF4F839BE4
:1004F00002C0DF91EBCF2F930F931F9300B32FEF29
:1005000003FB20F94F933F9310B34FEF012703FBF9
:1005100021F93BE031C04E7F012F10B3216028C08C
:10052000102F4D7F2260000000B329C04B7F246054
:10053000012F000010B32BC010B3477F28602AC0E2
:100540004F7E00B320612CC04F7D10B320622FC0BE
:100550004F7B00B3206432C0422700B349934FEF72
:100560000000102713FB20F910B31C70C9F1297F7C
:1005700091F2012703FB21F900B3237F89F2315067
:1005800058F1102713FB22F910B3277E79F20127C7
:1005900003FB23F92F7C81F200B3102713FB24F90E
:1005A0002F7971F200C010B3012703FB25F92F73D7
:1005B00059F200C000B3102713FB26F9223040F295
:1005C00000C010B3012703FB27F9243028F64F772A
:1005D000206810B30000F9CF10E41ABF00271CC038
:1005E0003B503195C31BD04010E41ABF0881033C37
:1005F00011F10B3401F120918B001981110F1213AD
:10060000EDCF4A81441F093659F10D3211F0013EF8
:1006100029F74F7009F0042F009392003F914F91FA
:100620001F910F912F91DF91CAB7C6FD4CCFCF918B
:10063000CFBFCF91189520919200222379F310918A
:100640009000112369F534306AF1309390002093C3
:100650008C0010918D003BE0311B30938D0022C047
:10066000009190000130E4F40AE54F7049F43091B4
:10067000600034FD19C000936000C4E7D0E018C0EA
:1006800030917F0034FD10C000937F00C0E8D0E0BF
:100690000FC02795A8F45150A9F4220F0000F9CFFC
:1006A0004AE503C042ED01C0432FC4E1D0E032E08F
:1006B00011B31C60939A11BB02B320E41CE05F935A
:1006C000012756E002BB279520F4515021F4220F58
:1006D000F9CF012756E000003B5A02BBD0F2279524
:1006E00028F4515029F4220F0000F9CF012756E0D9
:1006F000279502BB20F4515021F4220FF9CF012796
:1007000056E02991332302BB21F6037F109191001B
:10071000110FC651D04002BB11F010938B0010E4B2
:100720001ABF086011B3137F402F437F5F9100C051
:1007300000C002BB11BB42BB71CFFB01982F929549
:100740009F709A3008F0995D5D9BFECF905D9CB9DB
:100750008F708A3008F0895D5D9BFECF805D8CB91B
:100760005D9BFECF8AE38CB920E219C05D9BFECF72
:100770002CB99081892F82958F708A3008F0895D1D
:100780005D9BFECF805D8CB9892F8F708A3008F019
:10079000895D5D9BFECF3196805D8CB941504423CD
:1007A00029F75D9BFECF8DE08CB95D9BFECF8AE083
:1007B0008CB90895FC018381813041F488E990E08F
:1007C00090938F0080938E0082E108958AEA90E0F2
:1007D00090938F0080938E0085E60895FC0185B389
:1007E00091E0892785BBE0818E2F8076803221F4CD
:1007F000E7FD02C0909373008FEF0895FC0185B36D
:1008000092E0892785BB10821182128213821482A2
:100810001582168287E0089585B394E0892785BB09
:1008200081E0089585B390E2892785BB089587709C
:1008300087B987B187B9369A3699FECF24B135B1D9
:10084000C90108953F924F925F926F927F928F926B
:100850009F92AF92BF92CF92DF92EF92FF920F934F
:100860001F93DF93CF93CDB7DEB768970FB6F89499
:10087000DEBF0FBECDBFDE011996E2E6F0E080E1FB
:1008800001900D928150E1F72EE088E190E00FB6E3
:10089000F894A89581BD0FBE21BD83EF82BB11BA2C
:1008A0008C9894988C9A949A86E886B98FEF88BB36
:1008B00017BA85BB84BB539A86E289B90E94A70008
:1008C000109273007894DD24CC2410E03324339408
:1008D0007E010894E11CF11CFBE04F2EE0EB5E2E44
:1008E00070E4672E69E0762E50E9852E4FE7942E4E
:1008F00038E0A32E20E8B22EA8950E94EB0036B374
:1009000090E021E0963011F495E003C09D3009F4A9
:100910009CE0822F832319F4092F045C06C09E5F9C
:100920009E3010F4220FEECF00E0D01611F0CC2450
:10093000C39480917F0084FFDFCFCC2081F185B309
:10094000862585BBDD2011F460E005C0A982BA824E
:10095000DB821C8264E00023D1F0F701E60FF11D79
:100960007082862F8F5FF701E80FF11D80828F5F05
:10097000F701E80FF11D00838F5FF701E80FF11D0C
:1009800090826C5F683019F43092730002C010924C
:100990007300C7010E94B400D02ECC24ADCF812FAC
:1009A000877087B987B187B9369A3699FECF24B157
:1009B00035B1E12FF0E0EE0FFF1FEE0DFF1D80853A
:1009C0009185821B930B07960F97B0F085B38058E3
:1009D00085BB3187208749825A821A5B1B83165454
:1009E00083E0359527958A95E1F72C831092730063
:1009F000C70164E00E94B4001F5F183008F47CCF88
:080A000010E07ACFF894FFCF5B
:100A08005AFFFFFFFFFFFFFFFFFFFFFFFFFFFFFF93
:020A1800FFFFDE
:00000001FF
